:100000006F00C00413000000130000001300000084
:100010001300000013000000130000001300000094
:10002000F32E003093FE0E08638A0E00B72E0000F8
:10003000938E0E8073900E3073002030F32E1034A8
:10004000938E4E0073901E3473002030130E1000F8
:100050003705001093054006130650069306600608
:100060002320D5002F26B518130710006318E62E9D
:10007000032705006394E62E130E200037050010B9
:100080001305450093057006130680069306900637
:100090002320D5002F26B518130710006310E62C77
:1000A00003270500639CE62A130E30003705001075
:1000B0001305450093057006130680069306900607
:1000C0002F26B51813071000631AE628032705002A
:1000D0006396E628130E40003705001013058500CF
:1000E0009305A0061306B0069306C0062320D5008C
:1000F000AF2705102F26B5186392D7266310062662
:1001000003270500639CE524130E500037050010FB
:10011000130585009305D0061306E0069306F00646
:100120002320D5002F26B518631A062203270500C1
:100130006396E522130E6000370500101305C50015
:1001400093050007130610079306200737040010D5
:10015000130404019304300713094007930950075F
:100160002320D50023203401AF270510AF2A041027
:100170002F26B5182F2994186392D71E6310061ED8
:1001800003270500639CE51C639A3A1D6318091C4C
:10019000032A04006394441D130E700037050010F9
:1001A0001305450193058007130690079306A007E2
:1001B000930E00012320D500AF2705102F26B51878
:1001C000639ED718631C0618032705006398E5187B
:1001D000938EFEFF13054500938535001306360008
:1001E00093863600E3980EFC130E8000370500104E
:1001F0001305850193058007130690079306A00752
:10020000832705002F26B518130710006318E6147E
:10021000032705006394E714130E900037050010C0
:10022000130505109305B0071306C0079306D00702
:100230002320D500AF270510730000002F26B51826
:1002400013071000631CE610032705006398E610EF
:10025000130EA00037050010130505203708001005
:10026000130848209305E0071306F00793060008DB
:10027000930810082320D50023201801AF27081069
:100280002F26B51813071000631AE60C0327080081
:100290006396E80C130EB000370500101305053007
:1002A0009305200813063008930640082320D50044
:1002B000B71E0000938E0E8073904E30930E800018
:1002C000AF27051073900E301300000013000000DC
:1002D00013000000130000001300000013000000D2
:1002E0002F26B51813071000631AE606032705002A
:1002F0006396E606130EC00037050010130505408F
:100300009305C0081306D0089306E0082320D50003
:10031000B71E0000938E0E8073904E30B72E0000F3
:10032000938E8E80AF27051073900E30130000005F
:100330001300000013000000130000001300000071
:10034000130000002F26B518130710006318E600ED
:10035000032705006394E6006F000001370110F0E9
:10036000130141F22320C101370110F0130101F202
:100370002320010013000000130000001300000000
:0C03800013000000130000001300000038
:040000030000004CAD
:00000001FF
